:0200000480007A
:100000006F008004732F2034930F80006308FF0378
:10001000930F90006304FF03930FB0006300FF038E
:10002000130F000063040F0067000F00732F2034CC
:1000300063540F006F00400093E19153171F0000BD
:1000400023223FFC6FF09FFF732540F163100500F2
:10005000970200009382020173905230735000188F
:10006000970200009382020273905230B702008020
:100070009382F2FF7390023B9302F0017390023A75
:1000800097020000938282017390523073502030A7
:1000900073503030735040309301000097020000DD
:1000A000938282F673905230130510001315F501F8
:1000B000634C05000F00F00F930110009308D0056A
:1000C0001305000073000000970200009382020BEA
:1000D000638E020073905210B7B2000093829210A8
:1000E0007390223073232030E39862F47350003011
:1000F0003715000013050580732005301305200215
:1001000073203530970200009382420173901234BD
:10011000732540F173002030930120001303800009
:100120009302001073B00210970200009382020144
:1001300073901214730020109301100073000000DC
:100140006F008000631030020F00F00F6380010029
:100150009391110093E111009308D00513850100DC
:10016000730000000F00F00F930110009308D005FA
:100170001305000073000000F3222014E39662FCD4
:10018000970300009383C3FBF3221014E39E72FADB
:100190006FF05FFD731000C0000000000000000061
:1001A000000000000000000000000000000000004F
:1001B000000000000000000000000000000000003F
:1010000000000000000000000000000000000000E0
:1010100000000000000000000000000000000000D0
:1010200000000000000000000000000000000000C0
:1010300000000000000000000000000000000000B0
:081040000000000000000000A8
:040000058000000077
:00000001FF
